S02200006F70656E626C745F6E75636C656F5F73746D33326631303372622E7372656343
S3150800000000500020A90400088D0400088F04000889
S3150800001091040008930400089504000800000000F5
S31508000020000000000000000000000000970400081F
S3150800003099040008000000009B0400089D040008BD
S31508000040F1040008F1040008F1040008F1040008AE
S31508000050F1040008F1040008F1040008F10400089E
S31508000060F1040008F1040008F1040008F10400088E
S31508000070F1040008F1040008F1040008F10400087E
S31508000080F1040008F1040008F1040008F10400086E
S31508000090F1040008F1040008F1040008F10400085E
S315080000A0F1040008F1040008F1040008F10400084E
S315080000B0F1040008F1040008F1040008F10400083E
S315080000C0F1040008F1040008F1040008F10400082E
S315080000D0F1040008F1040008F1040008F10400081E
S315080000E0F1040008F1040008F1040008000000000B
S315080000F000000000000000000000000000000000F2
S3110800010000000000000000005FF808F195
S3150800010C10B5054C237833B9044B13B10448AFF337
S3150800011C00800123237010BD100000200000000091
S3150800012C1C1A000808B5034B1BB103490348AFF367
S3150800013C008008BD00000000140000201C1A0008EE
S3150800014C08B501F0CFF908BD08B501F0D9F908BD15
S3150800015C08B5054B9B6813F4005F01D1002008BD58
S3150800016C00F03CF80120FAE70010014008B56420BD
S3150800017C00F006F808BD08B500F008F808BD000040
S3150800018C014B1880704700BF2C00002008B501F001
S3150800019C5BF90E4B1B6898420FD30D4B1B786BB94A
S315080001AC0B4B01221A700B4B20221A6101F04CF9E9
S315080001BC094B1B881844054B186008BD044B0022D4
S315080001CC1A70044B20225A61F0E700BF3000002059
S315080001DC2E000020000801402C000020014B202294
S315080001EC5A6170470008014030B589B00024049460
S315080001FC0594069407941C4B9A6942F010029A616E
S3150800020C9A6902F010020192019A9A6942F0200248
S3150800021C9A619A6902F020020292029A9A6942F04D
S3150800022C04029A619B6903F004030393039B0F4D25
S3150800023C22462021284600F059FC4FF4005304931B
S3150800024C0594069404A90A4800F064FB2023049339
S3150800025C0123059306940223079304A9284600F064
S3150800026C59FB09B030BD00BF001002400008014020
S3150800027C0010014030B58FB00024079408940994F7
S3150800028C0A940B940C940D9405940694224BDA69F3
S3150800029C42F40032DA61DA6902F400320192019A08
S315080002AC9A6942F004029A619B6903F0040300936D
S315080002BC009B40F2044302930923039303230493FC
S315080002CC164D02A9284600F06FFC40F60803029367
S315080002DC0423039302A9284600F066FC4FF4E13385
S315080002EC0793089409940A940C230B930C940D9475
S315080002FC0B4C07A9204600F065FD236923F49043AF
S3150800030C2361636923F02A036361E36843F40053AA
S3150800031CE3600FB030BD00BF00100240000801407A
S3150800032C0044004008B5264A136823F0070343F037
S3150800033C02031360224B1B6803F00703022BF9D147
S3150800034C204B1A6842F480221A601A6842F48032EA
S3150800035C1A601C4B1B6813F4003FFAD0194A5368F1
S3150800036C23F47C1343F4E8135360136843F0807347
S3150800037C1360144B1B6813F0007FFAD0114B5A68A4
S3150800038C22F0F0025A605A6822F4E06242F4806263
S3150800039C5A605A6822F460525A605A6822F003026C
S315080003AC42F002025A60074B5B6803F00C03082BF9
S315080003BCF9D1054800F06CFD002000F0A5F808BD41
S315080003CC002002400010024000A24A0408B500F0C2
S315080003DCC1F8FFF7A7FFFFF707FFFFF74BFFFFF77C
S315080003ECAFFEFFF7B1FEFCE782B0104B9A6942F0FC
S315080003FC01029A619A6902F001020092009ADA697E
S3150800040C42F08052DA61DB6903F080530193019B59
S3150800041C074A536823F0E06343F0806353605368DC
S3150800042C23F0E063536002B0704700BF001002402F
S3150800043C0000014008B500F02FFC0E4800F05CFBEC
S3150800044C0D4800F059FB0D4BDA6922F40032DA61DB
S3150800045C9A6922F010029A619A6922F004029A614A
S3150800046CDA6922F08052DA619A6922F001029A61FD
S3150800047C08BD00BF001001400008014000100240F2
S3150800048C7047FEE7FEE7FEE7FEE7704770477047E2
S3150800049C08B500F071F808BD70470000002103E0AC
S315080004AC0B4B5B58435004310A480B4B42189A4283
S315080004BCF6D30A4A02E0002342F8043B084B9A4258
S315080004CCF9D3FFF7E9FF01F07FFAFFF77FFF7047D3
S315080004DC9C1A0008000000201000002010000020C4
S315080004EC48050020FEE7000010B5064B4FF0FF321A
S315080004FCDA6000241C61DA60DC60FFF79BFF20469B
S3150800050C10BD00BF0010024010B504460E4B1878FB
S3150800051C4FF47A73B3FBF0F30C4A1068B0FBF3F0A4
S3150800052C00F07CF868B90F2C01D901200AE00022EA
S3150800053C21464FF0FF3000F03DF8054B1C600020BB
S3150800054C00E0012010BD00BF0400002000000020C0
S3150800055C0800002008B5074A136843F01003136017
S3150800056C032000F015F80020FFF7CEFFFFF73CFF3D
S3150800057C002008BD00200240034A1168034B1B7873
S3150800058C0B441360704700BF2005002004000020B0
S3150800059C074AD36823F4E0631B041B0C000200F41F
S315080005ACE060184340F0BF6040F40030D0607047FC
S315080005BC00ED00E030B4174BDB68C3F30223C3F13C
S315080005CC0704042C28BF04241D1D062D18D9033B2B
S315080005DC4FF0FF3505FA04F421EA0401994005FAAF
S315080005EC03F322EA0303194300280BDB0901C9B2FA
S315080005FC00F1604000F5614080F8001330BC70478C
S3150800060C0023E5E700F00F000901C9B2024B1954A3
S3150800061CF4E700BF00ED00E014ED00E00138B0F19E
S3150800062C807F0AD2064B5860064AF02182F82310BE
S3150800063C0020986007221A6070470120704700BF97
S3150800064C10E000E000ED00E0044B0022DA61044AF9
S3150800065C136943F0010313610180704728050020D4
S3150800066C002002401A4BDB6813F0100F27D0194AEA
S3150800067CD36943F00203D3611023154AD26812F0EA
S3150800068C040F06D01349CA6942F00102CA6143F045
S3150800069C04030F4AD26912F0010F09D00D49CA6931
S315080006AC42F00402CA610A49CA6922F00102CA6107
S315080006BC40F20112934204D0054AD36070470023D6
S315080006CCDBE7034AD36923F00103D361704700BF04
S315080006DC00200240280500200A4B1B6913F0800FE6
S315080006EC0DD0084B084A5A6002F188325A601B69C9
S315080006FC13F0800F01D001207047002070470020AE
S3150800070C704700BF0020024023016745034A13695E
S3150800071C43F0800313610020704700BF002002409D
S3150800072C38B5044600F098FE0546174BDB6813F0FF
S3150800073C010F0AD0B4F1FF3FF7D00CB300F08CFED2
S3150800074C401BA042F1D9032019E00F4BDB6813F0CC
S3150800075C200F02D00C4B2022DA600B4BDB6813F00F
S3150800076C100F09D1084BDB6913F0010F04D1064BA6
S3150800077CDB6813F0040F05D0FFF774FF012038BDB2
S3150800078C0320FCE70020FAE7002002402DE9F84395
S3150800079C234C247E012C41D01E4690460F46044617
S315080007AC1F4B01221A764CF25030FFF7B9FF03465D
S315080007BC70BB012C29D0022C24D04FF0040900243C
S315080007CC4C4525D22101C1F12002A1F1200328FABA
S315080007DC01F106FA02F2114326FA03F3194389B218
S315080007EC07EB4400FFF730FF4CF25030FFF798FF49
S315080007FC0C4B1D6925F001051D61034640B90134F2
S3150800080CE4B2DDE74FF00209D9E74FF00109D6E764
S3150800081C034A002111761846BDE8F8830223FAE745
S3150800082C2805002000200240064B0022DA61064B00
S3150800083C1A6942F004021A611A6942F040021A61F6
S3150800084C704700BF2805002000200240064B0022F6
S3150800085CDA61064B1A6942F002021A6158611A6982
S3150800086C42F040021A617047280500200020024019
S3150800087C264B1B7E012B46D070B50E460446234BE1
S3150800088C01221A760368022B20D04CF25030FFF75F
S3150800089C47FF90BB4FF0FF333360A5680122E16830
S315080008ACA36803EB8123AB4228D92846FFF7CEFF72
S315080008BC4CF25030FFF734FF154A136923F0020344
S315080008CC13610246B8B905F58065E8E74CF2503075
S315080008DCFFF726FF08B1012210E00120FFF7A4FF5D
S315080008EC4CF25030FFF71CFF024609490B6923F0FE
S315080008FC04030B6102E0356000E00122034B002182
S3150800090C1976104670BD022210467047280500203D
S3150800091C00200240F0B482B000263246A2E0002D38
S3150800092C5AD0012D00D1CE68FF2B69D88446FF2BEF
S3150800093C69D89500DCF800400F27AF4024EA070475
S3150800094C06FA05F52C43CCF800404C6814F0805F89
S3150800095C00F087805F4CA56945F00105A561A4697F
S3150800096C04F001040194019C9508AF1C5A4C54F8E8
S3150800097C274002F00307BF004FF00F0C0CFA07FCD8
S3150800098C24EA0C0C554CA04243D004F58064A042D2
S3150800099C00F0818004F58064A0427ED004F5806462
S315080009ACA04234D0042435E04D4FBD4214D00BD9A7
S315080009BC4C4FBD4210D007F58037BD420CD0A7F579
S315080009CC8017BD42B0D107E0A7F58017BD4203D00A
S315080009DC07F58037BD42A7D18D687DB1012D08D0AA
S315080009EC44610826A0E7CE6808369DE7CE680C3623
S315080009FC9AE70461082697E7002695E7042693E705
S31508000A0C00F1040C93E7A2F10805AD0092E7032464
S31508000A1C00E00024BC4044EA0C0402352E4F47F88B
S31508000A2C25404C6814F4803F39D02F4D2C681C4354
S31508000A3C2C604C6814F4003F37D02B4D6C681C4363
S31508000A4C6C604C6814F4801F35D0274DAC681C4379
S31508000A5CAC604C6814F4001F33D0234DEC68234368
S31508000A6CEB6001320B6833FA02F430D0012494405F
S31508000A7C23409C42F5D14D68122DB7D094D8022D3F
S31508000A8CB1D07FF64CAF032DB6D0112D7FF44CAFF9
S31508000A9CCE68043648E70124BCE70224BAE7124DAF
S31508000AAC2C6824EA03042C60C3E70F4D6C6824EA0F
S31508000ABC03046C60C5E70C4DAC6824EA0304AC600F
S31508000ACCC7E7094DEC6824EA0303EB60C9E702B0F3
S31508000ADCF0BC7047001002400000014000080140BD
S31508000AEC00002110000031100004014012B909045D
S31508000AFC0161704701617047264B98420DD0264B11
S31508000B0C984216D0254B98421FD0254B984228D090
S31508000B1C244B984231D00120704703F58433DA68A8
S31508000B2C42F00402DA60DA6822F00402DA60002085
S31508000B3C704703F58233DA6842F00802DA60DA683D
S31508000B4C22F00802DA600020704703F58033DA6871
S31508000B5C42F01002DA60DA6822F01002DA6000203D
S31508000B6C704703F57C43DA6842F02002DA60DA68EB
S31508000B7C22F02002DA600020704703F57843DA6821
S31508000B8C42F04002DA60DA6822F04002DA600020AD
S31508000B9C704700BF00080140000C014000100140DE
S31508000BAC0014014000180140F0B50E68C6F30F2674
S31508000BBC96FAA6F5B5FA85F532E0A5F108024FF0D6
S31508000BCC0113934043F0806336E08C6893FAA3F7DD
S31508000BDCB7FA87F7BF004FF0030E0EFA07F722EAAB
S31508000BEC070293FAA3F7B7FA87F7BF00BC4022436C
S31508000BFC40F80C20CC6893FAA3F7B7FA87F7BF002E
S31508000C0C4FF0040E0EFA07F722EA070293FAA3F33B
S31508000C1CB3FA83F39B009C40224340F80C20013521
S31508000C2C36FA05F335D00123AB403342F7D0072DFE
S31508000C3CC3D840F20113AB400C69C7681A0A27EAF5
S31508000C4C020792FAA2F2B2FA82F204FA02F23A43D2
S31508000C5CC2604F684FEA136C50F80C4093FAA3F233
S31508000C6CB2FA82F292004FF00F0E0EFA02F224EA52
S31508000C7C020493FAA3F2B2FA82F2920007FA02F28B
S31508000C8C224340F80C204C68012C9ED0092CC6D166
S31508000C9C9BE70020F0BD0000184A136843F00103D7
S31508000CAC1360164B1B6813F0020FFAD0134A5368DD
S31508000CBC23F003035360114B5B6813F00C0FFAD146
S31508000CCC0E4A136823F0807313600C4B1B6813F0E1
S31508000CDC007FFAD1094B002058601A6822F450227A
S31508000CEC1A601A6822F0F80242F080021A609860BC
S31508000CFC5A6A42F080725A62704700BF001002406E
S31508000D0C034B5B68C3F30313024AD35CD8407047A2
S31508000D1C00100240341A0008034B5B68C3F3022325
S31508000D2C024AD35CD840704700100240441A0008A7
S31508000D3C034B5B68C3F3C223024AD35CD8407047A3
S31508000D4C00100240441A00080B4B5B6803F480330E
S31508000D5C7BB1094B5868C0F340400130074BB3FBD5
S31508000D6CF0F0054B5B68C3F38343023300FB03F0D7
S31508000D7C70470348F5E700BF0010024000127A00DE
S31508000D8C00093D0008B5054B5B6803F00C03082BFE
S31508000D9C02D1FFF7D9FF08BD0148FCE70010024055
S31508000DAC00127A0010B50446FFF7ECFF2060FFF737
S31508000DBCA7FF6060FFF7B0FFA0606068FFF7B8FF99
S31508000DCCE06010BDC36813F4005F01D001207047C2
S31508000DDC30B585B00D460446C36823F4B05323F0EA
S31508000DEC0C034A68C9680A4329690A431343C36052
S31508000DFCAB68026922F44052134303616B6942697A
S31508000E0C22F44072134343616846FFF7CBFF1C4B31
S31508000E1C9C4208D01B4B9C422AD01B4B9C4229D087
S31508000E2C012005B030BD039B33B32A6832B303EBFC
S31508000E3C830303EB83039200B3FBF2F3134DA5FB79
S31508000E4C03204009020191B2642202FB10321301FD
S31508000E5C3233A5FB0323C3F34F1303F0F0020A4402
S31508000E6C92B203F00F0313449BB2A3600020D8E799
S31508000E7C029BD9E7029BD7E70120D2E70120D0E7EE
S31508000E8C0038014000440040004800401F85EB51E3
S31508000E9C014B1860704700BF0000002072B67047FF
S31508000EAC62B6704708B5FFF7F9FF08BD10B500F034
S31508000EBCD1F900B910BDFFF74BF90028FAD000F0AC
S31508000ECC4FFBFFF711FB00F095FA00F0C7F920F07D
S31508000EDC604020F07F00044B986000F0BFF944682E
S31508000EECFFF7DEFFA047E5E700ED00E070B508E088
S31508000EFC4D1C461C0B78037000F066FB30462946E1
S31508000F0C2246531E9CB2002AF2D170BD08B5C1F315
S31508000F1C080353B903688B4209D040F8041B4FF4F5
S31508000F2C0072FFF7E3FF012000E0002008BD012056
S31508000F3CFCE72DE9F0410746FFF7CEFB00247F2C92
S31508000F4C14D83E68A30006EB03083B445D6800F022
S31508000F5C3BFB2A46002341460220FFF717FC38B90B
S31508000F6C56F82430AB4209D10134E8E7012400E0F5
S31508000F7C0024FFF7CBFB2046BDE8F0810024F8E7F8
S31508000F8C38B50D460C4B984211D004460B4B99427A
S31508000F9C07D1094C29462046FFF7B8FF48B1204629
S31508000FAC38BDFFF7C6FF0028F4D10024F7E7044C38
S31508000FBCF0E70024F3E700BF380200200020000801
S31508000FCC340000202DE9F04106460C4617461D460E
S31508000FDC21F4FF7828F001080368B3F1FF3F07D026
S31508000FEC336843450BD13368E41A3444043415E0AA
S31508000FFC4146FFF78BFF03460028F1D11FE0414617
S3150800100C3046FFF7BDFF06460028ECD1002316E054
S3150800101C17F8013B04F8013B013D0FD000F0D4FA58
S3150800102C331DE31AB3F5007FF2D308F50071304689
S3150800103CFFF7A6FF064628B1041DE9E70123184663
S3150800104CBDE8F0810023FAE74FF0FF33024A13603C
S3150800105C024A1360704700BF340000203802002093
S3150800106C10B54B1E114C241AA34218D8104B984293
S3150800107C17D90B18013B0D4CA34214D80B46014645
S3150800108C20F4FF7020F001000A4CA04203D00A4855
S3150800109CFFF798FF04E00948FFF794FF00E00020EB
S315080010AC10BD0020FCE70020FAE700BFFFFF01088F
S315080010BCFF1F00080020000834000020380200201A
S315080010CC30B587B0002305934A1E1F4B1B1A9A424C
S315080010DC31D820F47F7323F003031C4A93422ED98C
S315080010EC0A18013A184CA2422BD8C01A0144C1F36B
S315080010FC8F25C1F3090109B10135ADB2002401945C
S3150800110C039301230493FFF7E7FAA5420DD900F0E0
S3150800111C5BFA05A901A8FFF7ABFB50B9039B03F5CE
S3150800112C806303930134A4B2EFE70124FFF7EEFAC8
S3150800113C02E00024FAE70024204607B030BD00245C
S3150800114CFAE70024F8E700BFFFFF0108FF1F0008B5
S3150800115C104B1B68B3F1FF3F1AD000B583B00D4A8C
S3150800116C536891680B44D1680B4411690B44516957
S3150800117C0B4491690B44D26913445B4202AA42F8A8
S3150800118C043D04210448FFF76BFF03B05DF804FB2C
S3150800119C01207047380200200C2100080D4B1B68F3
S315080011AC0D4A12681A440D4B1B6813440C4A1268F4
S315080011BC13440C4A12681A440B4B1B681A440B4B03
S315080011CC1B6813440A4A1268DA4201D00020704799
S315080011DC0120704700200008042000080820000899
S315080011EC0C200008102000081420000818200008FD
S315080011FC0C21000808B50D4B1B68B3F1FF3F0BD14A
S3150800120C0B4B1B68B3F1FF3F0DD00948FFF791FE56
S3150800121C034648B1012307E00448FFF78AFE034654
S3150800122C0028EDD100E00123184608BD380200203D
S3150800123C34000020004870470020000808B5FFF766
S3150800124C03FF08BD08B5FFF70BFF08BD08B5FFF788
S3150800125C37FF08BD08B5FFF7A1FF08BD08B5FFF7AE
S3150800126CE9FF08BD08B5FFF773FF034608B918462A
S3150800127C08BDFFF7BFFF0346F9E70000054B1B68DF
S3150800128C13F0200F04D0034B5B68037001207047E2
S3150800129C002070470044004010B5094B586000F018
S315080012ACD3F800F10A04064B1B6813F0800F05D11E
S315080012BC00F08AF900F0C8F8A042F4D910BD00BFB6
S315080012CC0044004010B588B0104CE36823F4005372
S315080012DCE3604FF461430193002302930393049351
S315080012EC0C220592069301A92046FFF76BFD23698C
S315080012FC23F490432361636923F02A036361E3684B
S3150800130C43F40053E36008B010BD00BF004400402E
S3150800131C70B506460D46402904D82846FFF7BCFF8B
S3150800132C00240BE06F21074800F09AF8F5E700F067
S3150800133C4BF9305DFFF7B0FF0134A4B2ABB2A34250
S3150800134CF5D870BD4C1A000870B5254B1C78BCB97D
S3150800135C2448FFF793FF012801D0204670BD214B86
S3150800136C1B78013BDBB23F2BF7D800F06DF81E4B10
S3150800137C18601E4B00221A70194B01221A70ECE7E2
S3150800138C06460D46194B1B78013316481844FFF7C9
S3150800139C75FF0446012815D1144B1A780132D2B2BE
S315080013AC1A70104B1B789A4201D00024D5E71049C5
S315080013BC3046FFF79BFD0A4B00221A700B4B1B7825
S315080013CC2B70CAE700F040F8074B1B686433984249
S315080013DC03D90024024B1C70BFE70024BDE700BFED
S315080013EC7D0400203C040020800400207E0400209C
S315080013FC3D040020024B00221A605A609A6070471E
S3150800140C10E000E008B5FFF7F5FF054B054A5A60F2
S3150800141C00229A6005211960034B1A6008BD00BFAB
S3150800142C10E000E03F19010084040020044B1B68FF
S3150800143C13F4803F03D0034A1368013313607047D3
S3150800144C10E000E08404002008B5FFF7EFFF014B1D
S3150800145C186808BD8404002008B5FFF7F5FF08BD19
S3150800146C08B500F0B1F8FCE708B500F0A1F80128BA
S3150800147C03D00B4B1B78012B00D008BDFFF7E4FFFC
S3150800148C084B1B68084A1268134403F5FA7398420A
S3150800149CF3D3034B00221A70FFF708FDEDE700BFE4
S315080014AC8C040020880400209004002008B5054B05
S315080014BC1B78012B00D008BDFFF7C6FF024B18603E
S315080014CCF9E700BF8C0400209004002008B5044BF3
S315080014DC01221A70FFF7EAFFFFF7C6FF08BD00BF27
S315080014EC8C04002008B5FFF7DDFC00F069F8FFF75F
S315080014FC89FFFFF7A3FE00F00DF8FFF7E7FF08BD1D
S3150800150C08B500F061F8FFF791FF00F00FF8FFF748
S3150800151CABFF08BD08B500F0C5F9FFF7D3FE024BC3
S3150800152C00221A7008BD00BF0C00002000B583B05D
S3150800153C0DF107010848FFF707FF012802D003B091
S3150800154C5DF804FB054B00221A709DF8071002483B
S3150800155C00F0C8F9F3E700BF940400200C00002043
S3150800156C7047000008B5054B1B7813B100F0B2F9AB
S3150800157C08BDC9B2FFF7CCFEF8E700BF0C00002087
S3150800158C044B1B78013B022B01D9402070470020E5
S3150800159C704700BF0C000020044B1B78013B022B44
S315080015AC01D9402070470020704700BF0C0000206E
S315080015BC08B500F085F9034600B10123184608BDA5
S315080015CC08B5FEF7D3FD08BD08B5FEF7D4FD08BD72
S315080015DC014B00225A707047D4040020034BFE229C
S315080015ECDA7018710222A3F844207047D40400203C
S315080015FC10B5054C00232370FFF7EAFFFF23E370B1
S3150800160C0123A4F8443010BDD4040020064BFF2255
S3150800161CDA7000221A71597859719A71DA711A723C
S3150800162C0622A3F844207047D404002008B50020ED
S3150800163CFFF7D4FF08BD0000074BFF22DA70074AF4
S3150800164C9A6400221A715A719A710722C3F80720F4
S3150800165C0822A3F844207047D40400208C1A0008EA
S3150800166C044BFF22DA7042689A640122A3F84420DC
S3150800167C704700BFD404002008B53120FFF7AEFF31
S3150800168C08BD000038B5084CFF23E370002525710A
S3150800169C6571FFF775FFA071E571257265720723F1
S315080016ACA4F8443038BD00BFD404002038B5FFF781
S315080016BC8FFF0E4C01252570FF23E3701023237131
S315080016CC00236371FFF75CFFA071FFF765FFE071FC
S315080016DCFFF762FFC0F3072020726572A572082314
S315080016ECA4F84430FFF7AAFD38BD00BFD404002087
S315080016FC38B505464478FFF743FF0138844210DCB9
S3150800170C0A4C6A78A16C201DFFF7F0FBFF23E370E7
S3150800171C6A78A36C1344A3646B780133A4F8443039
S3150800172C38BD2220FFF75AFFFAE700BFD404002081
S3150800173C38B504464578FFF723FF0138854211DC96
S3150800174C61680A4DA9646278281DFFF7CFFBFF2351
S3150800175CEB706278AB6C1344AB6463780133A5F811
S3150800176C443038BD2220FFF739FFFAE7D4040020AD
S3150800177CF8B505461746002406E015F8013B1C4447
S3150800178CE4B2FFF721FF31464E1E0029F5D13C6025
S3150800179C0120F8BD10B5084CFF23E370E21D416823
S315080017ACA06CFFF7E5FF207100236371A371082372
S315080017BCA4F8443010BD00BFD404002038B5054643
S315080017CC0D4B9C6CFFF7DCFE6A1C411E2046FFF78E
S315080017DC39FD60B1084CFF23E370FFF7D1FE0138E1
S315080017ECA36C0344A3640123A4F8443038BD312008
S315080017FCFFF7F4FEFAE700BFD404002038B5044618
S3150800180C4578FFF7BDFE023885420EDC114BFF22E8
S3150800181CDA700122A3F84420617851B9FFF722FD4A
S3150800182C30B93120FFF7DAFE02E02220FFF7D6FEA8
S3150800183C38BDA21C074B986CFFF704FD28B16178DC
S3150800184C044A936C0B449364F2E73120FFF7C6FE07
S3150800185CEEE700BFD404002008B54168074B986C26
S3150800186CFFF7F4FC30B1054BFF22DA700122A3F81E
S3150800187C442008BD3120FFF7B1FEFAE7D404002056
S3150800188C08B5FFF713FB034BFF22DA700122A3F806
S3150800189C442008BDD404002008B589B2FFF762FEBF
S315080018AC08BD0000054B00221A709A6483F8432081
S315080018BCA3F844209A705A70704700BFD4040020CD
S315080018CC034B1B780BB1012070470020704700BFF3
S315080018DCD4040020024B002283F84320704700BF33
S315080018ECD404002008B50378FF2B04D0354A1278A7
S315080018FC012A14D008BDFFF7D9FE324B93F84330B2
S3150800190C012B5AD02F4BB3F944100029F2DD184697
S3150800191C012380F843300330FFF7BEFFEAE7C93BE3
S3150800192C352B46D8DFE803F03345454245453F3667
S3150800193C3C39454545454545454545454545454552
S3150800194C454545454545454545454545454545452D
S3150800195C4545241E1B2145454527452A2D30FFF7AD
S3150800196CC7FECAE7FFF7E4FEC7E7FFF779FEC4E749
S3150800197CFFF710FFC1E7FFF75FFEBEE7FFF756FE5E
S3150800198CBBE7FFF743FEB8E7FFF732FEB5E7FFF70D
S3150800199C15FFB2E7FFF732FFAFE7FFF773FEACE7C9
S315080019ACFFF75AFFA9E7FFF76BFFA6E7FFF764FEF9
S315080019BCA3E72020FFF712FE9FE71020FFF70EFE85
S315080019CCA0E700BFD404002070B500250C4E0D4CC2
S315080019DCA41BA410A54209D100F01AF800250A4E3A
S315080019EC0A4CA41BA410A54205D170BD56F8253087
S315080019FC98470135EEE756F8253098470135F2E752
S31508001A0C941A0008941A0008941A0008981A0008E0
S31508001A1CF8B500BFF8BC08BC9E467047F8B500BFC1
S30D08001A2CF8BC08BC9E46704791
S31508001A34000000000000000001020304060708096C
S31508001A440000000001020304433A2F576F726B2FFC
S31508001A54736F6674776172652F4F70656E424C5466
S31508001A642F5461726765742F536F757263652F41BE
S31508001A74524D434D335F53544D333246312F7273AF
S31508001A843233322E630000004F70656E424C5400A8
S30908001A943101000806
S30908001A980D01000826
S31508001A9C0024F400010000001000000004000000FF
S705080004A945
